:100000000C9424030C943F030C943F030C943F0383
:100010000C943F030C943F030C94E9110C943F03A0
:100020000C943F030C943F030C943F030C94C412B4
:100030000C943F030C943F030C943F030C943F0338
:100040000C943F030C943F030C943F030C943F0328
:100050000C943F039006E106220E09072A08460881
:100060007108E50825096509A509D409F409230AD9
:10007000430A9A0ACB0A1D0B480B750BAB0BAB0B53
:10008000AB0BAB0BAB0BAB0BAB0BAB0B6D0D750B32
:10009000A30DCD0D0672652C0375223B59781EBA4F
:1000A000E07A633BF47C75FF4E7E3172117F000075
:1000B000000005813504F483200001836246328309
:1000C000200000816246307F0000000582778C4F5F
:1000D00081432CE28217BF2483A48DD981E1D8A16A
:1000E00080DB67823E0634062A06200616060C06CA
:1000F0000206F805EE05E405DA05D005C605B105EA
:100100009C05870572055D05480533051E05090533
:10011000F404DF04CA04B504A204920480046B044E
:10012000660461045C04570452044C044604400411
:100130003A0434042E0424041A0410040604FC03B4
:10014000F003E403D803CC03C003B403AA03A00361
:100150008B0385037F03790373036D0367036103D7
:100160005B0355034F03490343033D033703310347
:100170002B0323031B0313030B030303FB02F302F1
:10018000EB02E302DB02D302CB02C302BB02B302E7
:10019000AB02960281026C0257024D024302390201
:1001A0002F021A020502FB01F101E001CB01B601A9
:1001B00000000000000053494420373A20766F7257
:1001C0006C7B756669676520462E00534944203371
:1001D0003A207065726D616E656E746520462E0002
:1001E00053696E6420536965207369636865723F63
:1001F000004E2D416E74722E2030004E2D416E74D3
:10020000722E2031004E6562656E616E7472696592
:10021000623A20617573202020004E6562656E6130
:100220006E74726965623A2065696E20202000490B
:10023000534F3134323330460049534F3134323327
:1002400030530049534F2039313431530049534F13
:100250002039313431460049534F20313432333064
:10026000206661737420696E6974200049534F20C1
:10027000313432333020736C6F7720696E697420AB
:100280000049534F203931343120392E3630302057
:1002900042617564200049534F2039313431203197
:1002A000302E3430302042617564004234205332A5
:1002B0003A200042342053313A2000423320533256
:1002C0003A200042332053313A2000423220533248
:1002D0003A200042322053313A200042312053323A
:1002E0003A200042312053313A2000423220533428
:1002F0003A200042322053333A2000423220533217
:100300003A200042322053313A2000423120533407
:100310003A200042312053333A20004231205332F8
:100320003A200042312053313A20005642345332B1
:100330000056423453310056423353320056423352
:100340005331005642325332005642325331005636
:100350004231533200564231533100564232533407
:100360000056423253330056423253320056423224
:100370005331005642315334005642315333005604
:1003800042315332005642315331004B65696E653C
:1003900020556E74657273747E747A756E67210071
:1003A0004B65796279746573200049534F2031346D
:1003B0003233300020423A4F322053656E732E00A4
:1003C00020423A53797320466C74200020423A440C
:1003D000726976696E67200020423A436C7364202C
:1003E0004C70200020423A4F70656E204C70200007
:1003F00020423A6E6F74207573656400413A4F3243
:100400002053656E7300413A53797320466C740033
:10041000413A44726976696E6700413A436C73648D
:10042000204C7000413A4F70656E204C70002042A5
:100430003A4F320020423A73460020423A4472005A
:1004400020423A634C0020423A6F4C0020423A4E20
:100450004100413A4F3200413A734600413A4472FA
:1004600000413A634C00413A6F4C00426974746534
:100470002054617374652064727E636B656E2E0018
:10048000446973706C617920616E70617373656E1D
:1004900021006765727B7420676566756E64656EA2
:1004A0002E004E65756573204D6F746F72737465A1
:1004B0007565722D004A4F42442C20454F42442C12
:1004C000204F42442049492020004A4F4244207591
:1004D0006E6420454F424420202020202020004AE6
:1004E0004F424420756E64204F42442049492020E9
:1004F000202020004A4F424420284A6170616E2922
:10050000202020202020202000454F42442C204F36
:1005100042442C204F424420494920202000454F8E
:10052000424420756E64204F424420202020202029
:10053000202000454F424420756E64204F424420E5
:100540004949202020202000454F4244202845755D
:10055000726F70612920202020202020006E6963A6
:100560006874204F4244206B6F6D706174696265DE
:100570006C004F42442049202020202020202020B1
:10058000202020202020004F424420756E64204F00
:100590004244204949202020202020004F4244206E
:1005A000284665646572616C2045504129202020F1
:1005B000004F424449492043616C69666F726E691D
:1005C0006120415242004A4F4244202B452B3200C9
:1005D0004A4F424420454F4244004A4F4244202B58
:1005E000322020004A4F4244202020202000454F46
:1005F0004244202B312B3200454F4244204F42448D
:100600002000454F4244202B32202000454F4244D9
:100610002020202020006B65696E204F424420007E
:100620004F42442D3120202020004F4244204F4291
:10063000442D32004F4244202020202020004F42F1
:10064000442D32202020200011241FBECFE5D4E00D
:10065000DEBFCDBF13E0A0E6B0E0ECEDF1E302C0F9
:1006600005900D92A231B107D9F713E0A2E1B3E0F2
:1006700001C01D92A138B107E1F70C9458120C94F7
:100680000000CF93DF93AC0120E030E0A0EDB7E0B5
:10069000C0E0D0E0CD010197F1F72F5F3F4F421747
:1006A0005307C0F7DF91CF91089560E080E40E9486
:1006B000761361E081E10E94761361E081E10E949E
:1006C000761361E08FE10E94761361E08EE00E9474
:1006D000761361E084E00E94761361E084E00E947A
:1006E000761361E084E00E94761361E084E00E946A
:1006F000761360E088E40E94761361E08FE10E9447
:10070000761361E08BE10E94761361E08BE10E9439
:10071000761361E08BE10E94761361E08BE10E9429
:10072000761361E08FE10E94761361E08BE10E9415
:10073000761361E08FE10E94761360E080E50E940D
:10074000761361E08EE00E94761361E08AE00E94F9
:10075000761361E08EE00E94761361E080E00E94F3
:10076000761361E080E00E94761361E080E00E94F1
:10077000761361E080E00E94761361E080E00E94E1
:1007800076130E948D13089581E0809312030895DB
:10079000109212030895AF92BF92CF92DF92EF9220
:1007A000FF920F931F9326E820BD7C01002711279D
:1007B00044E0EE0CFF1C001F111F4A95D1F7A12C3D
:1007C00032E1B32E3AE7C32ED12CC601B501A80100
:1007D00097010E94B018DA01C9010197A109B10976
:1007E000892F9A2FAB2FBB2780BDC601B501A80169
:1007F00097010E94B018DA01C901815089B90E949D
:1008000060131F910F91FF90EF90DF90CF90BF90FA
:10081000AF9008950E946713899A8898919A88E802
:1008200093E10E944103919888EC90E00E9441037B
:10083000919A88EC90E00E944103919A88EC90E0B4
:100840000E944103919888EC90E00E9441039198A6
:1008500088EC90E00E944103919A88EC90E00E941D
:100860004103919A88EC90E00E944103919888ECB2
:1008700090E00E944103919888EC90E00E9441032F
:1008800082B392B3892B826082BB88EC90E00E9495
:10089000410312BE8099FECF85E083BF80E0809B3C
:1008A000FECF8099FECF8F5F8430C8F313BE80994E
:1008B00003C00000809BFDCF82B79927AA2797FD30
:1008C000A095BA2FBC01CD010E94BB16DC01CB0163
:1008D00020E034E244EF55E4BC01CD010E94C7158D
:1008E000DC01CB0120E030E040E85EE3BC01CD015B
:1008F0000E941717DC01CB0120E030E040E05FE30D
:10090000BC01CD010E941717DC01CB019C01AD0198
:1009100060E070E080E89FE30E94C715DC01CB0136
:10092000BC01CD010E949E16DC01CB019C018E56BC
:1009300098428536910538F480EA98E20E94CB030C
:1009400081E090E008952E5435422536310538F483
:1009500080E895E20E94CB0382E090E0089580E079
:1009600090E0089508951F93CF93DF93CDB7DEB73E
:1009700026970FB6F894DEBF0FBECDBF0E94671357
:10098000899A809115038823A9F50E940A04182FDB
:1009900084E190E00E944103809117039091180335
:1009A000892B41F10E9418138A830E9418138B83AC
:1009B0009A81983019F4883029F00CC0943951F498
:1009C000843941F4113019F41093150303C082E007
:1009D0008093150380911503882361F084E190E0F2
:1009E0000E9441038B8180950E9447130E94181337
:1009F0000E94181386E490E00E94410326960FB6E9
:100A0000F894DEBF0FBECDBFDF91CF911F91089547
:100A1000BF92CF92DF92EF92FF920F931F93CF93EB
:100A2000DF93CDB7DEB7A4970FB6F894DEBF0FBE45
:100A3000CDBF182FB62E6A01FF24EF2C0E94C803E9
:100A4000A89580911503813021F0809115038230A3
:100A5000B9F488E60E9447130E9418138AE60E94A0
:100A600047130E94181381EF0E9447130E94181326
:100A7000812F0E9447130E941813812F8D531AC093
:100A8000809115038330D0F081EC0E9447130E94BF
:100A9000181383E30E9447130E94181381EF0E94EA
:100AA00047130E941813812F0E9447130E941813A6
:100AB000812F8B510E9447130E94181386E490E007
:100AC0000E9441038091170390911803892B39F1FB
:100AD000A8950E9418130E9418130E9418130E94D0
:100AE000181302E00E941813182F0E941813282FC1
:100AF000812F9927982F8827820F911DEE2DFF2790
:100B0000EE0FFF1FEC0FFD1F81839283E3941123EF
:100B100009F42111F394015007FFE4CFCDCFA8953C
:100B20000E94C403EB2DFF27EE0FFF1FEC0FFD1FEC
:100B3000319780819181F601808391838F2D992750
:100B4000A4960FB6F894DEBF0FBECDBFDF91CF9154
:100B50001F910F91FF90EF90DF90CF90BF9008957D
:100B6000FF920F931F93CF93C82F8B01A8950E94DC
:100B7000C803C23010F0C03219F4E4E0FE2E1FC0EA
:100B80008C2F82508230B0F0CC30A1F0C03191F087
:100B9000C43181F0C53171F0C63161F0C73151F017
:100BA000C83141F0C93131F0CA3121F0CB3111F0F7
:100BB000CF3119F472E0F72E02C061E0F62E809179
:100BC0001503813021F0809115038230E1F488E62D
:100BD0000E9447130E9418138AE60E9447130E943E
:100BE000181381EF0E9447130E94181381E00E949E
:100BF00047130E9418138C2F0E9447130E9418134A
:100C00008C2F8C531FC080911503833048F182ECE8
:100C10000E9447130E94181383E30E9447130E9407
:100C2000181381EF0E9447130E94181381E00E945D
:100C300047130E9418138C2F0E9447130E94181309
:100C40008C2F89510E9447130E9418130E94181379
:100C50000E9418130E9418130E9418130E94181360
:100C6000FF2041F0CF2D0E941813F80181938F01CE
:100C7000C150C9F70E94181388EC90E00E9441030C
:100C80000E940F13A8950E94C4038F2D9927CF911E
:100C90001F910F91FF900895AF92BF92CF92DF9274
:100CA000EF92FF920F931F93CF93DF93CDB7DEB7F1
:100CB0006F970FB6F894DEBF0FBECDBFA82EB62E2D
:100CC00000E010E02AE52817C8F0BE01645E7F4FFF
:100CD0000E94B005823041F48C8D9927182F00278F
:100CE0008D8D080F111D0AC0813021F48C8D082FC5
:100CF000112704C0882311F40C94AA0ECA2CDD24F9
:100D0000EE24FF24F601E032F10510F00C94220EDF
:100D1000E65DFF4FEE0FFF1F0590F491E02D099463
:100D200080911503813071F4EAE9F1E085919491A5
:100D30008E01095F1F4FBC01C8010E945815C801F0
:100D40000E94A21380911503823071F4ECE9F1E066
:100D5000859194918E01095F1F4FBC01C8010E94CB
:100D60005815C8010E94A21380911503833071F4B5
:100D7000EEE9F1E0859194918E01095F1F4FBC016E
:100D8000C8010E945815C8010E94A2138091150342
:100D9000843071F4E0EAF1E0859194918E01095F6D
:100DA0001F4FBC01C8010E945815C8010E94A21320
:100DB00082E0B81611F00C94AA0E80E690E00C9434
:100DC000470E8C8DE82FFF27813820F08F010058C7
:100DD000104001C08F01C801AA2797FDA095BA2F26
:100DE0007C018D0191E0B91651F42B2D43E0C8012F
:100DF000B7010E94F21384E690E00C94A80E8BE6F3
:100E000090E00E94A21321E043E0C801B7010C94D6
:100E1000420EC8018070A1E0BA1609F08EC07801B8
:100E20008C01B1E080309B0729F4E0E2F1E085918C
:100E3000949122C08050924029F4E2E2F1E0859141
:100E400094911AC084E00030180729F4E4E2F1E03C
:100E50008591949111C098E00030190729F4E6E2D9
:100E6000F1E08591949108C0A0E100301A0779F46F
:100E7000E8E2F1E0859194918E01095F1F4FBC017A
:100E8000C8010E945815C8010E94A2130FC08DE727
:100E900090E00E94A213C801AA2797FDA095BA2F3F
:100EA00020E043E0BC01CD010E94F21387011070E5
:100EB0000115110529F4EAE2F1E08591949107C04A
:100EC0000130110571F4ECE2F1E0859194918E010D
:100ED000095F1F4FBC01C8010E945815C8010C943E
:100EE000A80E0230110529F4EEE2F1E0859194910B
:100EF000EECF0430110529F4E0E3F1E085919491FF
:100F0000E6CF0830110529F4E2E3F1E085919491F0
:100F1000DECF0031110529F4E4E3F1E085919491ED
:100F2000D6CF8FE790E00E94A213C801AA2797FDB1
:100F3000A095BA2F20E043E0A3C678018C01B1E070
:100F400080309B0729F4E6E3F1E08591949107C096
:100F50008050924069F4E8E3F1E0859194918E012C
:100F6000095F1F4FBC01C8010E945815C8012CC061
:100F700084E00030180729F4EAE3F1E085919491C8
:100F8000EECF98E00030190729F4ECE3F1E0859109
:100F90009491E5CFA0E100301A0729F4EEE3F1E0E7
:100FA00085919491DCCF82E890E00E94A213C80161
:100FB000AA2797FDA095BA2F20E043E0BC01CD0100
:100FC0000E94F21386E890E00E94A213870110703D
:100FD0000115110529F4E0E4F1E08591949177CFB2
:100FE0000130110529F4E2E4F1E0859194916FCF8D
:100FF0000230110529F4E4E4F1E08591949167CF82
:101000000430110529F4E6E4F1E0859194915FCF75
:101010000830110529F4E8E4F1E08591949157CF67
:101020000031110529F4EAE4F1E0859194914FCF64
:1010300088E890E00E94A213C801AA2797FDA09516
:10104000BA2F20E043E0BC01CD010E94F2138DE8ED
:1010500090E07EC6B1E0BB16B1F484E6089FC00103
:1010600011246FEF70E00E949D18CB01AA2797FD15
:10107000A095BA2F2B2D43E0BC01CD010E94F213A5
:1010800081E990E065C688E990E0F2C2085210401C
:1010900021E0B21689F4B801882777FD8095982F52
:1010A00017FF03C02B2D42E002C02B2D43E00E940E
:1010B000F21389EA90E04CC680EB90E00E94A21304
:1010C000B801882777FD8095982F17FF03C021E08E
:1010D00042E002C021E043E00E94F21380EC90E085
:1010E00037C6C801AA2797FDA095BA2F7C018D01AC
:1010F00091E0B91699F5C801B7010E94BB16DC0151
:10110000CB0120E030E040E053E4BC01CD010E947F
:101110007C15DC01CB0120E030E048EC52E4BC015E
:10112000CD010E941717DC01CB0120E030E040E048
:101130005CE3BC01CD010E941717DC01CB01BC01AF
:10114000CD010E949E16DC01CB012B2D43E0BC019A
:10115000CD010E94F21383EC90E0FAC58AEC90E096
:101160000E94A213C801B7010E94BB16DC01CB018B
:1011700020E030E040E053E4BC01CD010E947C154A
:10118000DC01CB0120E030E048EC52E4BC01CD01B1
:101190000E941717DC01CB0120E030E040E05CE367
:1011A000BC01CD010E941717DC01CB01BC01CD01B0
:1011B0000E949E16DC01CB0121E043E0BC01CD0181
:1011C0000E94F2138BED90E0C3C5C801AA2797FDDA
:1011D000A095BA2F7C018D0191E0B91699F5C8014F
:1011E000B7010E94BB16DC01CB0120E030E040E0FB
:1011F00053E4BC01CD010E947C15DC01CB0120E051
:1012000030E048EC52E4BC01CD010E941717DC012C
:10121000CB0120E030E040E05CE3BC01CD010E9466
:101220001717DC01CB01BC01CD010E949E16DC0129
:10123000CB012B2D43E0BC01CD010E94F2138DEDBB
:1012400090E086C584EE90E08BCFC801AA2797FD79
:10125000A095BA2F7C018D0191E0B91699F5C801CE
:10126000B7010E94BB16DC01CB0120E030E040E07A
:1012700053E4BC01CD010E947C15DC01CB0120E0D0
:1012800030E048EC52E4BC01CD010E941717DC01AC
:10129000CB0120E030E040E05CE3BC01CD010E94E6
:1012A0001717DC01CB01BC01CD010E949E16DC01A9
:1012B000CB012B2D43E0BC01CD010E94F21385EF41
:1012C00090E046C58CEF90E04BCFC801AA2797FD70
:1012D000A095BA2F7C018D0191E0B91699F5C8014E
:1012E000B7010E94BB16DC01CB0120E030E040E0FA
:1012F00053E4BC01CD010E947C15DC01CB0120E050
:1013000030E048EC52E4BC01CD010E941717DC012B
:10131000CB0120E030E040E05CE3BC01CD010E9465
:101320001717DC01CB01BC01CD010E949E16DC0128
:10133000CB012B2D43E0BC01CD010E94F2138DE0C7
:1013400091E006C584E191E00BCFA1E0BA16B1F4BB
:10135000C80102C0880F991FAA95E2F7800F911F5C
:10136000AA2797FDA095BA2F2B2D43E0BC01CD01F4
:101370000E94F21385E291E00E94A2138CE291E0B8
:101380000E94A213C801880F991F800F911FAA27DE
:1013900097FDA095BA2F21E043E0BC01CD010E944A
:1013A000F2138BE391E0D4C4C801AA2797FDA0955E
:1013B000BA2F7C018D0191E0B91649F42B2D43E041
:1013C000C801B7010E94F2138FE391E0C1C486E423
:1013D00091E00E94A21321E043E0C801B7010E94FE
:1013E000F21385E591E0B4C4A1E0BA16A1F4C801F6
:1013F00017FD03969595879595958795AA2797FD4F
:10140000A095BA2F2B2D44E0BC01CD010E94F21310
:1014100089E591E09DC48FE591E00E94A213C80187
:1014200017FD03969595879595958795AA2797FD1E
:10143000A095BA2F21E044E0BC01CD010E94F21337
:101440008DE691E085C4C801AA2797FDA095BA2F23
:101450007C018D0191E0B91649F42B2D43E0C801C0
:10146000B7010E94F21381E791E072C488E791E02E
:101470000E94A21321E043E0C801B7010E94F213C9
:1014800086E891E065C400581040A1E0BA1639F52D
:10149000C801AA2797FDA095BA2FBC01CD010E94D3
:1014A000BB16DC01CB0120E030E040E05FE3BC0193
:1014B000CD010E941717DC01CB018E010F5F1F4F7A
:1014C0002B2D45E0BC01CD010E940D168CE28C83D2
:1014D000CE0101960E94A2138BE891E039C480E905
:1014E00091E00E94A213C801AA2797FDA095BA2FE8
:1014F000BC01CD010E94BB16DC01CB0120E030E035
:1015000040E05FE3BC01CD010E941717DC01CB0175
:101510008E010F5F1F4F21E045E0BC01CD010E940D
:101520000D168CE28C83CE0101960E94A2138FE9E6
:1015300091E00EC4B1E0BB16B9F40832110524F0F5
:1015400081EA91E00E94A21308521040C801AA2724
:1015500097FDA095BA2F2B2D42E0BC01CD010E9432
:10156000F21383EA91E0F4C38AEA91E00E94A213A5
:101570000832110524F081EA91E00E94A21308527A
:101580001040C801AA2797FDA095BA2F21E042E09C
:10159000BC01CD01A1CDC801AA2797FDA095BA2F06
:1015A0007C018D0191E0B91611F5C801B7010E94C7
:1015B000BB16DC01CB012AE037ED43E25CE3BC0162
:1015C000CD010E941717DC01CB018E010F5F1F4F69
:1015D00022E046E0BC01CD010E940D168CE28C8316
:1015E000CE0101960E94A2138AEB91E0B1C38EEB6B
:1015F00091E00E94A213C801B7010E94BB16DC0152
:10160000CB012AE037ED43E25CE3BC01CD010E944F
:101610001717DC01CB018E010F5F1F4F22E046E060
:10162000BC01CD010E940D168CE28C83CE01019687
:101630000E94A2138CEC91E08BC3A1E0BA16B1F426
:1016400084E6089FC00111246FEF70E00E949D188E
:10165000CB01AA2797FDA095BA2F2B2D43E0BC0103
:10166000CD010E94F2138EEC91E072C385ED91E002
:101670000E94A21384E6089FC00111246FEF70E05E
:101680000E949D18CB01AA2797FDA095BA2F94CD53
:10169000B1E0BB16A9F40130110519F486EE91E012
:1016A00057C30230110519F480EF91E051C30430A3
:1016B000110519F48AEF91E04BC384E092E048C32E
:1016C0000130110519F48EE092E042C30230110599
:1016D00019F483E292E03CC30430110519F488E365
:1016E00092E036C38DE492E033C321E0B21619F4E0
:1016F00082E692E02DC38CE692E00E94A21342E0C3
:1017000050E0BE016F5F7F4FC8010E94331511E0AA
:10171000F12E8E010F5F1F4FF80101900020E9F7B5
:101720003997E017F107A1F080E30E949E13F3942C
:101730002F2D3327F80101900020E9F73197E01BA6
:10174000F10B88E090E08E1B9F0B8217930760F7E8
:10175000CE010196FDC281E0B81609F0BEC01C8D15
:10176000812F992787FD9095A92FB92FBC01CD0115
:101770000E94BB1617FF06C020E030E040E853E4AB
:101780000E947D152AE037ED43EA5BE30E941717BC
:10179000DC01CB018E010F5F1F4F22E044E0BC0152
:1017A000CD010E940D168CE28A83CE0101960E9423
:1017B000A21382E190E00E9420152A2D332785FF95
:1017C00046C02731310551F12831310554F4253116
:1017D0003105D1F026313105E4F42431310579F0B9
:1017E000B9C22931310521F129313105E4F02A311D
:1017F000310519F12B31310509F424C0ABC2E2E502
:10180000F1E08591949163CBE4E5F1E085919491C9
:101810005ECBE6E5F1E08591949159CBE8E5F1E006
:101820008591949154CBEAE5F1E0859194914FCB69
:10183000ECE5F1E0859194914ACBEEE5F1E08591FC
:10184000949145CBE0E6F1E08591949140CB27312E
:10185000310551F12831310554F425313105D1F0EC
:1018600026313105E4F42431310579F073C2293190
:10187000310521F129313105E4F02A31310519F121
:101880002B31310509F424C065C2E2E6F1E085910F
:1018900094911DCBE4E6F1E08591949118CBE6E6B6
:1018A000F1E08591949113CBE8E6F1E08591949174
:1018B0000ECBEAE6F1E08591949109CBECE6F1E0FC
:1018C0008591949104CBEEE6F1E085919491FFCA65
:1018D000E0E7F1E085919491FACA82E190E00E94FC
:1018E00020152A2D332785FF46C02731310551F1B8
:1018F0002831310554F425313105D1F02631310537
:10190000E4F42431310579F085C02931310521F124
:1019100029313105E4F02A31310519F12B31310536
:1019200009F424C077C0E2E7F1E08591949168C0A2
:10193000E4E7F1E08591949163C0E6E7F1E08591F9
:1019400094915EC0E8E7F1E08591949159C0EAE78F
:10195000F1E08591949154C0ECE7F1E08591949188
:101960004FC0EEE7F1E0859194914AC0E0E8F1E0E4
:101970008591949145C02731310551F128313105C8
:1019800054F425313105D1F026313105E4F4243108
:10199000310579F03FC02931310521F12931310577
:1019A000E4F02A31310519F12B31310509F424C055
:1019B00031C0E2E8F1E08591949122C0E4E8F1E0E1
:1019C000859194911DC0E6E8F1E08591949118C04D
:1019D000E8E8F1E08591949113C0EAE8F1E085919F
:1019E00094910EC0ECE8F1E08591949109C0EEE885
:1019F000F1E08591949104C0E0E9F1E08591949142
:101A00008E01095F1F4FBC01C8010E945815C80113
:101A10000E94A2131C8D812F992787FD9095A92FD5
:101A2000B92FBC01CD010E94BB1617FF06C020E0F4
:101A300030E040E853E40E947D152AE037ED43EAA8
:101A40005BE30E941717DC01CB018E010F5F1F4F74
:101A500022E044E0BC01CD010E940D16BCE2FB2E49
:101A6000FA82CE0101960E94A21389E792E00E94B9
:101A7000A2138D8D8F3F09F46DC199278058904036
:101A8000AA2797FDA095BA2FBC01CD010E94BB16D5
:101A9000DC01CB0120E030E048EC52E4BC01CD0198
:101AA0000E941717DC01CB0120E030E040E05CE34E
:101AB000BC01CD010E941717DC01CB018E010F5F25
:101AC0001F4F21E046E0BC01CD010E940D16FD82B2
:101AD000CE0101960E94A21375CB91E0B916B1F424
:101AE0000E30110544F4F801E00FF11FEE51FF4FE5
:101AF00085919491ECC98CE792E00E94A213C801F1
:101B0000AA2797FDA095BA2F2B2D9AC00E3011054C
:101B100044F4F801E00FF11FE450FF4F85919491D8
:101B2000D6C98CE792E00E94A213C801AA2797FDAC
:101B3000A095BA2F21E042E0BC01CD010E94F21332
:101B400082E892E005C1A1E0BA16B1F4A7E0EA2E5E
:101B5000F12CEC0EFD1E012B29F4E2EAF1E0859157
:101B6000949104C0E4EAF1E085919491BC01C7012D
:101B70000E945815C701ECC0F7E0EF2EF12CEC0ED7
:101B8000FD1E012B29F4E6EAF1E085919491EECF58
:101B9000E8EAF1E085919491E9CFB1E0BB1621F438
:101BA0008DE40E949E1304C080E992E00E94A2137B
:101BB00020E13EE0C801B9010E949D187B01161684
:101BC00017064CF4629FC001639F900D729F900DA9
:101BD0001124081B190BC701AA2797FDA095BA2F3E
:101BE00020E042E0BC01CD010E94F2138AE30E9492
:101BF0009E132CE330E0C801B9010E949D187B01BF
:101C0000161617064CF4629FC001639F900D729FD9
:101C1000900D1124081B190BC701AA2797FDA09549
:101C2000BA2F20E042E0BC01CD010E94F2138AE30A
:101C30000E949E13C801AA2797FDA095BA2F20E005
:101C400042E01EC08DE992E00E94A21320E042E033
:101C5000C701B6010E94F21321E0B21619F483EA1B
:101C600092E076C080E2A81681F086EA92E00E94B7
:101C7000A213C801AA2797FDA095BA2F21E045E03D
:101C8000BC01CD010E94F21365C08FEA92E00E9470
:101C9000A2138C8D40E150E0BE016F5F7F4F99270A
:101CA0000E9433158E010F5F1F4FF8010190002035
:101CB000E9F73297E017F10719F480E30E949E13C9
:101CC000C8010E946F150E94A2138D8D40E150E063
:101CD000B80199270E943315F80101900020E9F717
:101CE0003297E017F10719F480E30E949E13C801B0
:101CF0000E946F150E94A2138E8D40E150E0B80142
:101D000099270E943315F80101900020E9F73297D6
:101D1000E017F10719F480E30E949E13C8010E94A6
:101D20006F150E94A2138F8D40E150E0B8019927F2
:101D30000E943315F80101900020E9F73297E0176F
:101D4000F10719F480E30E949E13C8010E946F15E9
:101D50000E94A2136F960FB6F894DEBF0FBECDBFE0
:101D6000DF91CF911F910F91FF90EF90DF90CF9077
:101D7000BF90AF90089599278330910511F1843079
:101D800091054CF481309105A9F082309105BCF4A5
:101D9000892B69F0089585309105C1F08530910552
:101DA0009CF086309105A9F00797A9F0089561E0AD
:101DB000862F02C06BE081E00E94D413089561E099
:101DC00001C06BE082E0F8CF61E001C06BE083E02E
:101DD000F3CF61E001C06BE084E0EECFAF92BF9241
:101DE000CF92DF92EF92FF920F931F93CF93DF93E7
:101DF000CDB7DEB7C856D0400FB6F894DEBF0FBEE1
:101E0000CDBFBB24AB2C0E948D138B2D0E94BB0E2B
:101E10006B2D8DE00E9476130E94C403B099FECF13
:101E20007E010894E11CF11CF70193E6B92E119292
:101E3000BA94B7FEFCCF0E94C803BE016B597F4F16
:101E400080E00E94B0050E94C40320E0AE014B591F
:101E50005F4F31E000E810E0822F9927DC01A40FEA
:101E6000B51FFC0183E0EE0FFF1F8A95E1F7EE0D31
:101E7000FF1D319677E0B72E8C919927802391230F
:101E80008017910709F4308316950795BA94319617
:101E9000B7FEF2CF2F5F2430E8F281E08983BB24C4
:101EA000CC24DD2422E0A216C1F4C6019927869530
:101EB000979588278050904881F486010C0D1D1D50
:101EC00060E0C801805090400E94281560E0C80181
:101ED0008F5F9F4F0E942815BFC086010C0D1D1DEE
:101EE000C801805090400E942015E82EC8018F5FE5
:101EF0009F4F0E942015F82E8B2D0E94BB0EFF20B5
:101F000099F081E0F81661F4C601992786959795B6
:101F100088278050904821F481EA91E00E94A21322
:101F20006F2D8E2D0E944C068B2D0E94BB0E00E063
:101F300010E0B09B76C08AE090E00E944103B09927
:101F4000FECF81E0F81661F4C60199278695979532
:101F500088278050904811F0B2E0FB2EE39418C01F
:101F600082E0F81619F4A1E0FA2E12C0EE2081F4F6
:101F7000FF2099F4C6019927869597958827805068
:101F8000904819F4E1E0FE2E08C072E0F72E05C07B
:101F900083E68E1510F4FF24EF2C9E012F5F3F4F38
:101FA000F901EE0DF11D8081882339F4E39483E675
:101FB0008E15B0F7FF24EF2CF3CF22E0F21661F07C
:101FC000C60199278695979588278050904821F4D7
:101FD00081EA91E00E94A213EE2039F4FF2029F457
:101FE00085EB92E00E94A2130BC00E94C8036F2DE4
:101FF0008E2D0E944C060E94C40382E0F81661F008
:10200000C60199278695979588278050904821F09A
:102010008FEB92E00E94A2138B2D0E94BB0E00E07A
:1020200010E00F5F1F4F8AE090E00E94410381E0C3
:102030000139180708F47DCF86010C0D1D1D6E2D8A
:10204000C801805090400E9428156F2DC8018F5FF5
:102050009F4F0E942815AF2CB3940894C11CD11C2B
:1020600027E02B1508F01ECF0E94C80360E08CE02B
:102070000E9476130E948D13C859DF4F0FB6F89453
:10208000DEBF0FBECDBFDF91CF911F910F91FF90AB
:10209000EF90DF90CF90BF90AF900895AF92BF9236
:1020A000DF92EF92FF920F931F93CF93DF93CDB701
:1020B000DEB769970FB6F894DEBF0FBECDBFBE0185
:1020C0006A5E7F4F80E00E94B0050E94C403DD2459
:1020D0008D2D992736E1A32EB12CAC0EBD1E8C019F
:1020E0000A0D1B1D805F9F4F0E942015F8019081F3
:1020F000981709F47AC0E8E1F1E085919491BC0168
:10210000CE0101960E945815CE0101960E94A2139D
:1021100082E00E94BB13EAE1F1E085919491BC0159
:10212000CE0101960E945815CE0101960E94A2137D
:1021300083E00E94BB13ECE1F1E085919491BC0136
:10214000CE0101960E945815CE0101960E94A2135D
:1021500084E00E94BB13EEE1F1E085919491BC0113
:10216000CE0101960E945815CE0101960E94A2133D
:10217000B09BFECF8AE090E00E94410327E0D22E80
:1021800001E010E078010894E108F10860E0C7017F
:102190000E94281560E0C8010E942815DA9482E0A8
:1021A00090E0E80EF91E080F191FD7FEEFCF6E89D9
:1021B00080E190E00E942815F501618181E190E0C5
:1021C0000E942815F501628182E190E00E942815A5
:1021D000F501638183E190E00E9428150E948D1330
:1021E000B099FECF0E94EE0E05C0D394F3E0FD152A
:1021F00008F06ECF0E94C80369960FB6F894DEBF50
:102200000FBECDBFDF91CF911F910F91FF90EF9047
:10221000DF90BF90AF900895CF93DF93CDB7DEB737
:1022200065970FB6F894DEBF0FBECDBF60E08CE0BF
:102230000E94761384E00E94BB13809115038130C5
:1022400069F4E2E9F1E085919491BC01CE01019637
:102250000E945815CE0101960E94A2138091150389
:10226000823069F4E4E9F1E085919491BC01CE01FA
:1022700001960E945815CE0101960E94A2138091EA
:102280001503833069F4E6E9F1E085919491BC018E
:10229000CE0101960E945815CE0101960E94A2130C
:1022A00080911503843069F4E8E9F1E08591949117
:1022B000BC01CE0101960E945815CE0101960E94E4
:1022C000A21380ED97E00E9441030E948D13659652
:1022D0000FB6F894DEBF0FBECDBFDF91CF9108954A
:1022E000AF92BF92CF92DF92EF92FF920F931F9324
:1022F000CF93DF93CDB7DEB722970FB6F894DEBF4A
:102300000FBECDBFAA24A895B09B02C00E94EE0EBE
:10231000AE014F5F5F4F61E083E00E940805D82E59
:10232000AE014F5F5F4F61E087E00E940805D80E65
:10233000CC24EE24FF248C2D0E94BB0EDD2051F016
:10234000CC2041F481E0A8268A2D0E949E138BECBC
:1023500092E02CC087010E0D1F1DC80180509040D7
:102360000E942015B82EC8018F5F9F4F0E94201534
:10237000082F882391F0813061F4C7019927869551
:10238000979588278050904821F481EA91E00E9437
:10239000A213602F8B2D0E944C06002349F4DD20F0
:1023A00039F081E0C81621F485ED92E00E94A21375
:1023B000C3940894E11CF11C27E02C1508F0BBCF56
:1023C0000E94C40380EA9FE00E9441030E94C80368
:1023D0009ACF1F920F920FB60F9211241F932F9333
:1023E0003F934F935F936F937F938F939F93AF939D
:1023F000BF93EF93FF93CF93DF93CDB7DEB72297D1
:10240000DEBFCDBF1DBC1CBC80911203882399F098
:102410007894A89580911603982F8F5F8093160368
:10242000923048F0AE014F5F5F4F61E083E00E9461
:1024300008051092160310911503112309F58091D8
:1024400016038F5F809316038091160380FD03C0EF
:102450008EE20E949E13809116038C3088F01093B8
:1024600016030E94FA1480E797E10E94410388E175
:1024700090E028E00FB6F894A89581BD0FBE21BD6D
:102480002296F894DEBFCDBFDF91CF91FF91EF91FF
:10249000BF91AF919F918F917F916F915F914F917C
:1024A0003F912F911F910F900FBE0F901F90189585
:1024B000CFE5D4E0DEBFCDBF04B601FC06C004B654
:1024C00000FC03C004B602FE04C00E9401150E9475
:1024D000550304B603FE09C088E10FB681BD11BCE7
:1024E0000FBE0E94F0140E94FA14B8980E948D1337
:1024F00080EE92E00E94A21382E00E94BB1385EF5F
:1025000092E00E94A21384E00E94BB1387E093E054
:102510000E94A21304B601FC06C004B600FC03C06E
:1025200004B602FE04C080ED97E00E94410314BE91
:1025300082E19AE79BBD8ABD89B7806189BF84E04B
:102540008EBD789480911503882359F40E94B304BA
:10255000809115038823B1F3109216030E94F3149F
:10256000F1CF0E940C1188E190E02FE00FB6F894B3
:10257000A89581BD0FBE21BD0E944E100E94701112
:1025800080E090E00C94ED181F920F920FB60F921E
:1025900011242F933F935F936F937F938F939F9318
:1025A000AF93BF93EF93FF938CB1992790931C0344
:1025B00080931B038091170390911803C297F8F43E
:1025C00020911703309118038091190390911A03F9
:1025D000820F931F62E370E00E948918FC01EE0FE6
:1025E000FF1FE35EFC4F80911B0390911C038083CF
:1025F00091832F5F3F4F3093180320931703FF9170
:10260000EF91BF91AF919F918F917F916F915F916A
:102610003F912F910F900FBE0F901F901895109221
:102620001A031092190310921803109217030895B9
:102630008091170390911803892BD1F3F89480911E
:102640001703909118030197909318038093170331
:102650008091190390911A03FC01E80FF91FE35EC2
:10266000FC4F019690931A03809319030190F08117
:10267000E02D8091190390911A03C29720F01092D7
:102680001A031092190378948E2F99270895282FF2
:102690005D9BFECF80E29EE40197F1F72CB908958F
:1026A000CF93DF93EC0188810E94471388818823B0
:1026B00021F0219688818823E1F7DF91CF91089559
:1026C0000E940F137894539A549A579A08951AB8FF
:1026D0000E940F130895AD9A88EC90E00197F1F7EE
:1026E000AD9888EC90E00197F1F708951F93CF9390
:1026F000C82F662311F010E101C0162F8C2F829590
:102700008F70812B85BB0E946B13CF701C2B15BB68
:102710000E946B13CF911F91089560E0862F0E9455
:10272000761380E49FE10197F1F760E081E00E9479
:10273000761380E49FE10197F1F7089561E00E942C
:10274000761308951F93CF93DF93EC0110E08881F7
:10275000882369F0FE01E10FF11D80810E949E1324
:102760001F5FFE01E10FF11D8081882399F7DF9142
:10277000CF911F910895813019F460E080E809C07D
:10278000823019F460E080EA04C0833029F460E00C
:1027900080EC0E9476130895843021F460E080EE8E
:1027A0000E94761308950895962F813021F460E0F9
:1027B000892F81580BC0823021F460E0892F815627
:1027C00005C0833031F460E0892F81540E94761374
:1027D0000895843029F460E0892F81520E94761395
:1027E000089508959F92AF92BF92CF92DF92EF9299
:1027F000FF920F931F93CF935B016C01C42F90E363
:10280000992EC150222311F080E2982ED7FE0BC0E2
:102810008DE20E949E13D094C094B094A094A11C09
:10282000B11CC11CD11C80EAA81686E8B80681E05C
:10283000C80680E0D80664F0C601B50120EA36E893
:1028400041E050E00E94D218DA01C901805D03C066
:10285000C53018F0892D0E949E13C601B50120EAEB
:1028600036E841E050E00E94D2187B018C0180E103
:10287000A81687E2B80680E0C80680E0D80664F0B3
:10288000C801B70120E137E240E050E00E94D218D1
:10289000DA01C901805D03C0C43018F0892D0E949F
:1028A0009E13C801B70120E137E240E050E00E94EA
:1028B000D2187B018C0188EEA81683E0B80680E070
:1028C000C80680E0D80664F0C801B70128EE33E0FE
:1028D00040E050E00E94D218DA01C901805D03C0D7
:1028E000C33018F0892D0E949E13C801B70128EE4D
:1028F00033E040E050E00E94D2187B018C0184E676
:10290000A816B104C104D10464F0C801B70124E6DB
:1029100030E040E050E00E94D218DA01C901805D49
:1029200003C0C23018F0892D0E949E13C801B70160
:1029300024E630E040E050E00E94D2187B018C0198
:102940008AE0A816B104C104D10464F0C801B7013B
:102950002AE030E040E050E00E94D218DA01C901DC
:10296000805D03C0CC2319F0892D0E949E13C801FD
:10297000B7012AE030E040E050E00E94D218DC01CC
:10298000CB01805D0E949E13CF911F910F91FF900C
:10299000EF90DF90CF90BF90AF909F9008951F93DE
:1029A00013E015BB0E946B1380E991E00197F1F7EA
:1029B00015BB0E946B1380E991E00197F1F715BBFD
:1029C0000E946B1380E991E00197F1F760E082E0EB
:1029D0000E94761380E991E00197F1F71F91089525
:1029E0008FE384BB089560E08CE00E9476138F9A99
:1029F000979A089560E088E00E9476138F9A9798DE
:102A000008950E94F0148FE384BB80E49CE9019751
:102A1000F1F70E94CF1460E08CE20E94761360E030
:102A200089E00E94761360E088E20E9476130E949B
:102A3000F31460E086E00E9476130E948D130895DF
:102A4000E199FECF9FBB8EBBE09A99278DB3089585
:102A5000E199FECF9FBB8EBB6DBB0FB6F894E29A97
:102A6000E19A0FBE0895E62FF72F2E2F3F2FE894FF
:102A70004230CCF04532BCF44A3029F497FB1EF4C6
:102A8000909581959F4F642F77270E948918805DCC
:102A90008A330CF0895D8193862F972F009799F7E1
:102AA00016F45DE25193932F822F10820C945F15E0
:102AB000FB01DC0105900D920020E1F70895DC0197
:102AC000FC0101900020E9F73297AE17BF0730F400
:102AD0007C916081708331976D93F7CF0895DC010D
:102AE0005C91552341F05F7D51341CF05B350CF453
:102AF0005C931196F5CF08955058192E66D101D0E8
:102B000049C1BA176207730784079507B1F188F4C2
:102B10000EF410940B2EBA2FA02D062E622F202D0E
:102B2000072E732F302D082E842F402D092E952F20
:102B3000502DFF275523B9F0591B49F0573E98F007
:102B4000469537952795A795F0405395C9F776F0A8
:102B5000BA0F621F731F841F30F4879577956795AE
:102B6000B795F040939517FA0F2E0895BF1BBB271A
:102B7000BA0B620B730B840BF6CFDEF643C1592FF1
:102B8000482F372F262F9FE380E8772766271DD110
:102B900001D000C1552359F0992369F09F575F5721
:102BA000951B33F442F4903811F4915805C00AC1D2
:102BB00091589F3F09F426C1BB2711246217730760
:102BC000840730F4660F771F881FBB1F915098F35E
:102BD00011D00F920FD00F920DD0A0E82617370713
:102BE00048071B0609F0A048BA2F602D7F918F91EE
:102BF00000240895A0E80024621773078407B10534
:102C000028F0621B730B840BB1090A2A660F771F29
:102C1000881FBB1FA69581F70895DF93CF931F935D
:102C20000F93E8018C01000F111F1F3F31F49EE448
:102C300081E49993899399937AC04F9399231AF4D5
:102C40000DE209939F77022F03959F938F937F93B4
:102C50006F93622F7727882799270E94BB16906869
:102C6000AC019B0191E480E2772766270E946517FB
:102C70005FEF4FEF0E9404172F913F914F915F91AB
:102C80000E947D15102F013009F4002751E440E225
:102C900033272227621773078407950724F00E94C1
:102CA000C7151395F3CF9F938F937F936F930E94D4
:102CB0009E16562F505D59930E94BB162F913F913F
:102CC0004F915F910E947C15905851E440E2332768
:102CD00022270E941717101711F45EE259931A95D4
:102CE00011F718825F91EF91FF91FF93EF93452FBA
:102CF000442312F440954395CE01BF01861B970BE8
:102D0000142F181B90E284179CF455236AF0219627
:102D10003196E40FF11D83955A9152938A95E1F70C
:102D200092931A95E9F704C099931A95E9F71882D6
:102D30008F919F918C01CF91DF91089597FB51D096
:102D40009F3738F0FEE9F91B982F872F762F6B2FCE
:102D500005C055C09695879577956795F150D0F742
:102D60003EF490958095709561957F4F8F4F9F4F62
:102D70000895E89403C097FB0EF4F3DFB62F672F96
:102D8000782F892F9EE9002405C09A95BB0F661FF6
:102D9000771F881F11249923A1F08823B2F79F3F42
:102DA00059F0BB0F48F421F4002011F460FF04C077
:102DB0006F5F7F4F8F4F9F4F881F9795879597F92C
:102DC00008951DC09FEF80EC0895052E092607FA8F
:102DD000440F551F5F3F79F0AA27A51708F051E06F
:102DE0004795880F991F9F3F31F0BB27B91708F00F
:102DF00091E0879508959F919F911124E3CF6627D5
:102E0000772788279927089597FBEBDF992329F0E7
:102E10005F3F29F0552319F00AF4F1CFD3CF940F77
:102E2000151E01F4B7CF592F482F372F262FCDDF8E
:102E300001D0B0CF992339F0552329F09F575F5720
:102E4000950F13F4CAF1DECF91589F3FE1F3A62FFF
:102E500000241124BB2766275527F8E0A69520F407
:102E6000020E131EB41F651F220F331F441F551F70
:102E7000FA95A1F7F8E0E72F7727F8E0E69520F438
:102E8000130EB41F651F7A1F330F441F551FAA1F4F
:102E9000FA95A1F7F82F8827F69520F4B40F651F4F
:102EA0007A1F8E1F440F551FAA1FEE1FFF23A1F785
:102EB00088231AF4939539F485CF000C111CBB1F9D
:102EC000661F771F881F01280895552371F19923E4
:102ED00062F059F15F934F933F932F93BBD02F91A3
:102EE0003F914F915F91A3DF25C09F938F937F9375
:102EF0006F935F934F933F932F93952F842F732F4F
:102F0000622F1CDFF9DD91158105710561052F9197
:102F10003F914F915F916F917F918F919F9121F0A0
:102F20009F775058E2DF50584DCF9FE380E87727D6
:102F300066270895092E99234AF052E441EB32E7BF
:102F4000683173078407950758F03CCF9F7752E4A8
:102F50004EEA3CEA603573078407950708F04FCFC7
:102F60000F925FE348EB3AEA2BE361DFFF92EF92C7
:102F7000DF92CF9250E04CE096D0E4E9F0E01ED032
:102F80005F2D4E2D3D2D2C2DCF90DF90EF90FF909B
:102F9000FEE94595441F551FF51B5527406804C0A1
:102FA0004695379527955795FA95D2F7452F550FA2
:102FB000550B2ADF0F9007FCE2CD0895092E11DF93
:102FC000FF92EF92DF92CF92BF92AF92B02CC92EB8
:102FD000D82EE72EF62EA59018D0A590AA2071F035
:102FE0009F938F937F936F936F2D7E2D8D2D9C2DAF
:102FF0000CD02F913F914F915F91CCDDAF90BF905E
:10300000CF90DF90EF90FF90C5CE7ED047FB406819
:1030100004C02F2D3E2D4D2D5C2DEF93FF930ADF25
:10302000FF91EF9171D0AA2707F80B24102C0426EA
:1030300007FA4068FF9365DDFF91992341F08823EB
:1030400032F09A95BB0F661F771F881FF8CFAA949E
:1030500001F7089597FDB6CEC4DE992309F4B2CEE8
:10306000FF92EF92DF92CF92C92E9FE38F77E2EB30
:10307000F0E0A4DF0C2CC92ED82EE72EF62E602D02
:103080006E57770B872F972F76DE5FE341E332E7AA
:1030900028E1CDDE5C2D4D2D3E2D2F2DCF90DF90E4
:1030A000EF90FF902ACD97FB9CDECF93DF93D52F37
:1030B000C42F55274427332722279923D9F09F3738
:1030C000C8F0F92F67DE592F482F372F262FF639F2
:1030D00068F434DE50DEC030CD0721F06993799377
:1030E000899399939058DF91CF9107CD992788279D
:1030F00077276627C030CD0721F02993399349936C
:103100005993DF91CF9146CE5591459135912591B7
:103110000895AA1BBB1B51E107C0AA1FBB1FA6171E
:10312000B70710F0A61BB70B881F991F5A95A9F770
:1031300080959095BC01CD01089597FB092E072637
:103140000AD077FD04D0E5DF06D000201AF4709590
:1031500061957F4F0895F6F7909581959F4F08955B
:10316000A1E21A2EAA1BBB1BFD010DC0AA1FBB1F8B
:10317000EE1FFF1FA217B307E407F50720F0A21BFD
:10318000B30BE40BF50B661F771F881F991F1A946A
:1031900069F760957095809590959B01AC01BD0194
:1031A000CF01089597FB092E05260ED057FD04D0B8
:1031B000D7DF0AD0001C38F4509540953095219502
:1031C0003F4F4F4F5F4F0895F6F79095809570955C
:0C31D00061957F4F8F4F9F4F0895FFCFF8
:1031DC0020942000204665686C2E004665686C655E
:1031EC0072616E7A61686C3A2020202000410020C8
:1031FC004200413A20003F0020423A20003F20206C
:10320C0000254C61737420006265722E204C617332
:10321C0074776572743A20200002434B7E686C0010
:10322C004B7E686C6D697474656C3A2020202000AC
:10323C00024300254B45544231004B75727A2E45A2
:10324C00696E2E54722E20423120002500254C45EB
:10325C00544231004C616E672E45696E2E54722EAD
:10326C002042312000254B45544232004B75727A76
:10327C002E45696E2E54722E2042322000254C456C
:10328C00544232004C616E672E45696E2E54722E7C
:10329C0020423220006B5061204B64004B726166FF
:1032AC007473742E64722E3A2020006B5061006B84
:1032BC00706120456B004162732E64722E45696EFD
:1032CC006C2E3A20006B70610075706D20200044EC
:1032DC007265687A61686C3A202020200075706DE8
:1032EC00006B6D6820202000546163686F6D6574FD
:1032FC0065723A2020006B6D2F680002205A760010
:10330C005A7E6E64766F7265696C756E673A0002F0
:10331C0000200002434C7566740045696E2E4C7596
:10332C00667474656D702E3A2000674C6D004C7598
:10333C0066746D617373653A202020006700254424
:10334C00726F736C0044726F7373656C6B6C61702D
:10335C0070653A2020005A774C2E766F72672E00DB
:10336C005A774C2E6E6163682E005A774C2E204192
:10337C00757320005A774C2E206B2E412E005A77F5
:10338C006569746C7566743A20766F7267657363E1
:10339C00682E005A776569746C7566743A206E6194
:1033AC0063686765732E20005A776569746C75665F
:1033BC00743A20417573202020202020005A776514
:1033CC0069746C7566743A20756E62656B616E6EAD
:1033DC0074004F322053656E736F72004F3220535E
:1033EC00656E736F723A2020005620004F424420C5
:1033FC0023002020202020202020202020202000FE
:10340C004D6F746F7273746172743A20005049443A
:10341C0020230020200020576572743A20200020C1
:10342C0049443A2000202020202020202020002069
:10343C002020202020202020202000446961676E5D
:10344C006F736520002020202020202020202000C9
:10345C004F4244204949204C434420202020202026
:10346C00302E34310020207777772E626C616675B0
:10347C0073656C2E64650053756368652045435510
:02348C0020001E
:00000001FF
